:107800000C945D3C0C94953C0C947A3C0C947A3C22
:107810000C947A3C0C947A3C0C947A3C0C947A3C10
:107820000C947A3C0C947A3C0C947A3C0C947A3C00
:107830000C947A3C0C947A3C0C947A3C0C947A3CF0
:107840000C947A3C0C947A3C0C947A3C0C947A3CE0
:107850000C947A3C0C947A3C0C947A3C0C947A3CD0
:107860000C947A3C0C947A3C040309041C037700C2
:10787000770077002E0066006900730063006800DF
:107880006C002E00640065000E035500530042009A
:1078900061007300700012011001FF000008C016A3
:1078A000DC05020101020001090212000101008051
:1078B000FA09040000000000000011241FBECFEFF1
:1078C000D8E0DEBFCDBF11E0A0E0B1E0E8E9F0E82C
:1078D00002C005900D92A630B107D9F711E0A6E0DD
:1078E000B1E001C01D92AD33B107E1F70E94F33D55
:1078F0000C944A400C94003CA82FB92F80E090E0F3
:1079000041E050EA609530E009C02D9182279795BB
:10791000879510F084279527305EC8F36F5FA8F332
:107920000895EADF8D939D930895CF93CFB7CF93BA
:10793000C3954F9BE9F74F9B0BC04F9B09C04F9BD3
:1079400007C04F9B05C04F9B03C04F9B01C0D3C0D6
:107950000F92DF93C0912001DD27C95DDE4F012E1C
:107960004F9B03C0DF910F90E6CF2F930F931F9390
:107970004F932FEF4F6F09B107FB20F95F933F93B0
:1079800050E03BE065C019B10126502957FDC8956C
:1079900059B1012707FB25F92F7309B1B1F0502721
:1079A000102717FB26F909B02230F0F000C019B1FA
:1079B000012707FB27F90126502909B02430E8F5F3
:1079C0004F77206819B10000F6CF50274F7D206215
:1079D00009B0102F000000C009B10026502910275F
:1079E00017FB26F909B0E2CF4F7B09B1206400C034
:1079F000DACF01265029147809B069F14E7F216051
:107A0000012F19B128C0002650294D7F09B02260EE
:107A1000102F29C0012650294B7F09B02460012F67
:107A20002DC019B101265029477F2860000009B0F8
:107A30002EC04F7E09B1206130C0422709B1499361
:107A400000265029102709B04FEF17FB20F9297F96
:107A500019B179F2147859F10126502909B001279A
:107A600007FB21F9237F09B171F20026502931501B
:107A7000D0F009B0102717FB22F9277E19B151F277
:107A800001265029012707FB09B023F92F7C49F271
:107A9000000009B1102717FB24F90026502909B06E
:107AA0002F7939F270CF11E01CBB002717C03B5073
:107AB0003195C31BD04011E01CBB0881033CF9F099
:107AC0000B34E9F020911E011981110F1213EDCF33
:107AD000093651F10D3211F0013E39F700932501BD
:107AE0003F915F914F911F910F912F91DF910F90D7
:107AF000CCB3C0FD1DCFCF91CFBFCF9118952091B2
:107B00002501222369F310912301112321F534303B
:107B100022F13093230120931F01109120013BE0BB
:107B2000311B3093200119C00091230101309CF4D6
:107B30000AE53091000134FD11C000930001C3E15A
:107B4000D1E010C0052710E000C021C0052710E0DB
:107B5000C8950BB914C03AE501C032ED032EC0E060
:107B6000D0E032E01AB114685F9A0BB11AB954E848
:107B700020E84FEF20FF05270BB9279517951C3FED
:107B800028F700004552B0F720FF052727950BB9CD
:107B900017951C3FB8F629913A9561F70B7710912C
:107BA0002401110F0BB9C250D04011F010931E01E7
:107BB00011E01CBB00681AB11B77402F4B7754E0D3
:107BC0005A95F1F70BB91AB94BB98ACF1BB8F8948B
:107BD0001DBA1092690081E085BF15BEE0911101C8
:107BE000F091120109952F923F924F925F926F92FE
:107BF0007F928F929F92AF92BF92CF92DF92EF923D
:107C0000FF920F931F93CF93DF9388E10FB6F89401
:107C100080936000109260000FBE5F9A04B601FE70
:107C200021C214BE81E085BF82E085BF4F991AC290
:107C300080916900836080936900E89A4F9BFECF32
:107C400057987894E8E86E2EE8E77E2E7CE6472E7B
:107C500078E7572E68E6262E68E7362E58EAC52EB6
:107C600058E7D52E46E9A42E48E7B42E37E0832EF8
:107C700031E0932E90912301935097FD60C1809144
:107C800020012CE0E22EF12CE81AF10827E231E085
:107C9000E20EF31E80911F018D3209F0D9C0983099
:107CA00009F04BC133EC309313018AE58093000156
:107CB00010920B01D7013C91832F807611962C9165
:107CC0001197882309F452C09092220180922101D9
:107CD000233009F513969C91139714968C91149761
:107CE00012962C91203339F48370E82FF0E0EE5F88
:107CF000FE4F80810CC0203A19F40E94344007C026
:107D0000203C21F4F70165810E943C4080E0809393
:107D10000A0194E08AC0253011F491E086C0822FD8
:107D200084508630E0F4D70112968D919C91139780
:107D300090930D0180930C01293009F475C01696BB
:107D40009C91169790930E0115968C91827080935A
:107D50000F012093100137FD6EC02FEF6DC0223050
:107D600009F062C0B1E0B09306015EC0F701828104
:107D700010921C01222331F410921D012CE131E0FC
:107D800092E04DC0253019F48093240145C026307F
:107D900099F5D70113968C91813029F4B092220184
:107DA000A092210106C0823031F4D0922201C0920B
:107DB000210192E11DC08330D1F4F7018281882333
:107DC00031F4309222012092210194E011C08130DF
:107DD00031F450922201409221019CE109C082308D
:107DE00031F470922201609221019EE001C090E086
:107DF000F0E4F0930B0119C0283019F426E231E0C9
:107E000009C0293019F48093260106C02A3021F4D4
:107E10002CE131E091E003C02CE131E090E03093BF
:107E200022012093210101C090E0D70117968C9187
:107E3000882331F009C0292F80E880930B0105C009
:107E4000F7012681291708F0292F2093010175C019
:107E500080910B0187FF71C080910E01192F891746
:107E600008F4182F811B80930E0100E0882309F489
:107E700001E080911001873010F0E70115C05091AA
:107E80000F01E0910C01F0910D0140E04BC0809199
:107E90000C0190910D01019690930D0180930C01BE
:107EA000019769910E943C409E012E19211778F399
:107EB00040C0CF018F779070892B49F4F89433E05C
:107EC00030935700E895789407B600FCFDCF4E5FDD
:107ED000F894D7018D919D917D01B1E00C01B09393
:107EE0005700E895112478949F012E5F3F4FC901F8
:107EF0008F779070892B31F0002399F0411788F02B
:107F0000552379F0F89485E080935700E8957894AC
:107F100007B600FCFDCFF89491E190935700E895E7
:107F20007894F901411708F4C4CFF0930D01E09360
:107F30000C01002311F01092010110922301809195
:107F4000000184FF80C0809101018F3F09F47BC054
:107F5000182F893008F018E0811B8093010180916F
:107F6000130198E8892780931301112309F458C05D
:107F700080910B0187FF2BC080910E01811708F4BF
:107F8000182F811B80930E0100911001C4E1D1E0F4
:107F9000E12EFF24EC0EFD1E16C0E0910C01F091C5
:107FA0000D01073020F0CF010E94344001C08491C0
:107FB0008883219680910C0190910D0101969093F8
:107FC0000D0180930C01CE15DF0539F727C02091F4
:107FD00021013091220186FF0DC0A4E1B1E080E0D3
:107FE00090E0F901E80FF91FE491ED93019618175D
:107FF000C1F708C0D901912FE4E1F1E08D9181939F
:108000009150E1F71150812F90E01F5F0196820F90
:10801000931F909322018093210102C0193068F4CC
:1080200084E191E0612F0E94913C612F6C5F6C3084
:1080300041F08FEF8093010104C08FEF8093010125
:108040006EE16093000194E189B1847831F491503C
:10805000D9F71092240110921E0180910601882305
:1080600009F408CE0E94E63DF999FECF92BD81BD8C
:10807000F89A992780B50895262FF999FECF1FBA4F
:1080800092BD81BD20BD0FB6F894FA9AF99A0FBE41
:0880900001960895F894FFCF5A
:068098005AFF1E950F00C7
:040000030000780081
:00000001FF
